
15_uart_rx_interrupt.elf:     file format elf32-littlearm

Sections:
Idx Name          Size      VMA       LMA       File off  Algn
  0 .isr_vector   00000198  08000000  08000000  00010000  2**0
                  CONTENTS, ALLOC, LOAD, READONLY, DATA
  1 .text         000003f8  08000198  08000198  00010198  2**2
                  CONTENTS, ALLOC, LOAD, READONLY, CODE
  2 .rodata       00000000  08000590  08000598  00010598  2**0
                  CONTENTS, ALLOC, LOAD, DATA
  3 .ARM.extab    00000000  08000590  08000590  00010598  2**0
                  CONTENTS
  4 .ARM          00000000  08000590  08000590  00010598  2**0
                  CONTENTS
  5 .preinit_array 00000000  08000590  08000598  00010598  2**0
                  CONTENTS, ALLOC, LOAD, DATA
  6 .init_array   00000004  08000590  08000590  00010590  2**2
                  CONTENTS, ALLOC, LOAD, DATA
  7 .fini_array   00000004  08000594  08000594  00010594  2**2
                  CONTENTS, ALLOC, LOAD, DATA
  8 .data         00000000  20000000  20000000  00010598  2**0
                  CONTENTS, ALLOC, LOAD, DATA
  9 .bss          00000020  20000000  08000598  00020000  2**2
                  ALLOC
 10 ._user_heap_stack 00000600  20000020  08000598  00020020  2**0
                  ALLOC
 11 .ARM.attributes 00000030  00000000  00000000  00010598  2**0
                  CONTENTS, READONLY
 12 .debug_info   000015c7  00000000  00000000  000105c8  2**0
                  CONTENTS, READONLY, DEBUGGING, OCTETS
 13 .debug_abbrev 0000041e  00000000  00000000  00011b8f  2**0
                  CONTENTS, READONLY, DEBUGGING, OCTETS
 14 .debug_aranges 000000b8  00000000  00000000  00011fb0  2**3
                  CONTENTS, READONLY, DEBUGGING, OCTETS
 15 .debug_ranges 00000090  00000000  00000000  00012068  2**3
                  CONTENTS, READONLY, DEBUGGING, OCTETS
 16 .debug_macro  0000ec61  00000000  00000000  000120f8  2**0
                  CONTENTS, READONLY, DEBUGGING, OCTETS
 17 .debug_line   00000dbd  00000000  00000000  00020d59  2**0
                  CONTENTS, READONLY, DEBUGGING, OCTETS
 18 .debug_str    00053f6e  00000000  00000000  00021b16  2**0
                  CONTENTS, READONLY, DEBUGGING, OCTETS
 19 .comment      00000053  00000000  00000000  00075a84  2**0
                  CONTENTS, READONLY
 20 .debug_frame  000001d8  00000000  00000000  00075ad8  2**2
                  CONTENTS, READONLY, DEBUGGING, OCTETS

Disassembly of section .text:

08000198 <__do_global_dtors_aux>:
 8000198:	b510      	push	{r4, lr}
 800019a:	4c05      	ldr	r4, [pc, #20]	; (80001b0 <__do_global_dtors_aux+0x18>)
 800019c:	7823      	ldrb	r3, [r4, #0]
 800019e:	b933      	cbnz	r3, 80001ae <__do_global_dtors_aux+0x16>
 80001a0:	4b04      	ldr	r3, [pc, #16]	; (80001b4 <__do_global_dtors_aux+0x1c>)
 80001a2:	b113      	cbz	r3, 80001aa <__do_global_dtors_aux+0x12>
 80001a4:	4804      	ldr	r0, [pc, #16]	; (80001b8 <__do_global_dtors_aux+0x20>)
 80001a6:	f3af 8000 	nop.w
 80001aa:	2301      	movs	r3, #1
 80001ac:	7023      	strb	r3, [r4, #0]
 80001ae:	bd10      	pop	{r4, pc}
 80001b0:	20000000 	.word	0x20000000
 80001b4:	00000000 	.word	0x00000000
 80001b8:	08000578 	.word	0x08000578

080001bc <frame_dummy>:
 80001bc:	b508      	push	{r3, lr}
 80001be:	4b03      	ldr	r3, [pc, #12]	; (80001cc <frame_dummy+0x10>)
 80001c0:	b11b      	cbz	r3, 80001ca <frame_dummy+0xe>
 80001c2:	4903      	ldr	r1, [pc, #12]	; (80001d0 <frame_dummy+0x14>)
 80001c4:	4803      	ldr	r0, [pc, #12]	; (80001d4 <frame_dummy+0x18>)
 80001c6:	f3af 8000 	nop.w
 80001ca:	bd08      	pop	{r3, pc}
 80001cc:	00000000 	.word	0x00000000
 80001d0:	20000004 	.word	0x20000004
 80001d4:	08000578 	.word	0x08000578

080001d8 <main>:
static void uart_callback(void);
void USART2_IRQHandler(void);

char key;

int main(void){
 80001d8:	b580      	push	{r7, lr}
 80001da:	af00      	add	r7, sp, #0
	RCC->AHB1ENR |= GPIOAEN;
 80001dc:	4b0b      	ldr	r3, [pc, #44]	; (800020c <main+0x34>)
 80001de:	6b1b      	ldr	r3, [r3, #48]	; 0x30
 80001e0:	4a0a      	ldr	r2, [pc, #40]	; (800020c <main+0x34>)
 80001e2:	f043 0301 	orr.w	r3, r3, #1
 80001e6:	6313      	str	r3, [r2, #48]	; 0x30
	GPIOA->MODER |= (1U<<10);
 80001e8:	4b09      	ldr	r3, [pc, #36]	; (8000210 <main+0x38>)
 80001ea:	681b      	ldr	r3, [r3, #0]
 80001ec:	4a08      	ldr	r2, [pc, #32]	; (8000210 <main+0x38>)
 80001ee:	f443 6380 	orr.w	r3, r3, #1024	; 0x400
 80001f2:	6013      	str	r3, [r2, #0]
	GPIOA->MODER &= ~(1U<<11);
 80001f4:	4b06      	ldr	r3, [pc, #24]	; (8000210 <main+0x38>)
 80001f6:	681b      	ldr	r3, [r3, #0]
 80001f8:	4a05      	ldr	r2, [pc, #20]	; (8000210 <main+0x38>)
 80001fa:	f423 6300 	bic.w	r3, r3, #2048	; 0x800
 80001fe:	6013      	str	r3, [r2, #0]

	uart2_rx_inerrupt_init();
 8000200:	f000 f8ca 	bl	8000398 <uart2_rx_inerrupt_init>
	uart2_rxtx_init();
 8000204:	f000 f856 	bl	80002b4 <uart2_rxtx_init>

	while (1){
 8000208:	e7fe      	b.n	8000208 <main+0x30>
 800020a:	bf00      	nop
 800020c:	40023800 	.word	0x40023800
 8000210:	40020000 	.word	0x40020000

08000214 <uart_callback>:
	}
}

static void uart_callback(void){
 8000214:	b480      	push	{r7}
 8000216:	af00      	add	r7, sp, #0
	key = USART2->DR;
 8000218:	4b0d      	ldr	r3, [pc, #52]	; (8000250 <uart_callback+0x3c>)
 800021a:	685b      	ldr	r3, [r3, #4]
 800021c:	b2da      	uxtb	r2, r3
 800021e:	4b0d      	ldr	r3, [pc, #52]	; (8000254 <uart_callback+0x40>)
 8000220:	701a      	strb	r2, [r3, #0]
	if(key == '1'){
 8000222:	4b0c      	ldr	r3, [pc, #48]	; (8000254 <uart_callback+0x40>)
 8000224:	781b      	ldrb	r3, [r3, #0]
 8000226:	2b31      	cmp	r3, #49	; 0x31
 8000228:	d106      	bne.n	8000238 <uart_callback+0x24>
		GPIOA->ODR |= LED_PIN;
 800022a:	4b0b      	ldr	r3, [pc, #44]	; (8000258 <uart_callback+0x44>)
 800022c:	695b      	ldr	r3, [r3, #20]
 800022e:	4a0a      	ldr	r2, [pc, #40]	; (8000258 <uart_callback+0x44>)
 8000230:	f043 0320 	orr.w	r3, r3, #32
 8000234:	6153      	str	r3, [r2, #20]
			}
	else{
		GPIOA->ODR &= ~LED_PIN;
	}
}
 8000236:	e005      	b.n	8000244 <uart_callback+0x30>
		GPIOA->ODR &= ~LED_PIN;
 8000238:	4b07      	ldr	r3, [pc, #28]	; (8000258 <uart_callback+0x44>)
 800023a:	695b      	ldr	r3, [r3, #20]
 800023c:	4a06      	ldr	r2, [pc, #24]	; (8000258 <uart_callback+0x44>)
 800023e:	f023 0320 	bic.w	r3, r3, #32
 8000242:	6153      	str	r3, [r2, #20]
}
 8000244:	bf00      	nop
 8000246:	46bd      	mov	sp, r7
 8000248:	f85d 7b04 	ldr.w	r7, [sp], #4
 800024c:	4770      	bx	lr
 800024e:	bf00      	nop
 8000250:	40004400 	.word	0x40004400
 8000254:	2000001c 	.word	0x2000001c
 8000258:	40020000 	.word	0x40020000

0800025c <USART2_IRQHandler>:

void USART2_IRQHandler(void){
 800025c:	b580      	push	{r7, lr}
 800025e:	af00      	add	r7, sp, #0
	/*check if RXNE set*/
	if (USART2->SR & SR_RXNE){
 8000260:	4b04      	ldr	r3, [pc, #16]	; (8000274 <USART2_IRQHandler+0x18>)
 8000262:	681b      	ldr	r3, [r3, #0]
 8000264:	f003 0320 	and.w	r3, r3, #32
 8000268:	2b00      	cmp	r3, #0
 800026a:	d001      	beq.n	8000270 <USART2_IRQHandler+0x14>
		/*do someting*/
		uart_callback();
 800026c:	f7ff ffd2 	bl	8000214 <uart_callback>
	}
}
 8000270:	bf00      	nop
 8000272:	bd80      	pop	{r7, pc}
 8000274:	40004400 	.word	0x40004400

08000278 <__NVIC_EnableIRQ>:
  \details Enables a device specific interrupt in the NVIC interrupt controller.
  \param [in]      IRQn  Device specific interrupt number.
  \note    IRQn must not be negative.
 */
__STATIC_INLINE void __NVIC_EnableIRQ(IRQn_Type IRQn)
{
 8000278:	b480      	push	{r7}
 800027a:	b083      	sub	sp, #12
 800027c:	af00      	add	r7, sp, #0
 800027e:	4603      	mov	r3, r0
 8000280:	71fb      	strb	r3, [r7, #7]
  if ((int32_t)(IRQn) >= 0)
 8000282:	f997 3007 	ldrsb.w	r3, [r7, #7]
 8000286:	2b00      	cmp	r3, #0
 8000288:	db0b      	blt.n	80002a2 <__NVIC_EnableIRQ+0x2a>
  {
    NVIC->ISER[(((uint32_t)IRQn) >> 5UL)] = (uint32_t)(1UL << (((uint32_t)IRQn) & 0x1FUL));
 800028a:	79fb      	ldrb	r3, [r7, #7]
 800028c:	f003 021f 	and.w	r2, r3, #31
 8000290:	4907      	ldr	r1, [pc, #28]	; (80002b0 <__NVIC_EnableIRQ+0x38>)
 8000292:	f997 3007 	ldrsb.w	r3, [r7, #7]
 8000296:	095b      	lsrs	r3, r3, #5
 8000298:	2001      	movs	r0, #1
 800029a:	fa00 f202 	lsl.w	r2, r0, r2
 800029e:	f841 2023 	str.w	r2, [r1, r3, lsl #2]
  }
}
 80002a2:	bf00      	nop
 80002a4:	370c      	adds	r7, #12
 80002a6:	46bd      	mov	sp, r7
 80002a8:	f85d 7b04 	ldr.w	r7, [sp], #4
 80002ac:	4770      	bx	lr
 80002ae:	bf00      	nop
 80002b0:	e000e100 	.word	0xe000e100

080002b4 <uart2_rxtx_init>:
	/*enable uart module*/
	USART2 ->CR1 |= CR1_UE;

}

void uart2_rxtx_init(void){
 80002b4:	b580      	push	{r7, lr}
 80002b6:	af00      	add	r7, sp, #0
	/*********configure the uart gpioa pin*********/
	/*enable clock access to gpioa*/
	RCC->AHB1ENR |= GPIOAEN;
 80002b8:	4b33      	ldr	r3, [pc, #204]	; (8000388 <uart2_rxtx_init+0xd4>)
 80002ba:	6b1b      	ldr	r3, [r3, #48]	; 0x30
 80002bc:	4a32      	ldr	r2, [pc, #200]	; (8000388 <uart2_rxtx_init+0xd4>)
 80002be:	f043 0301 	orr.w	r3, r3, #1
 80002c2:	6313      	str	r3, [r2, #48]	; 0x30

	/*set PA2 mode to alternate function mode*/
	GPIOA->MODER &= ~(1U<<4);
 80002c4:	4b31      	ldr	r3, [pc, #196]	; (800038c <uart2_rxtx_init+0xd8>)
 80002c6:	681b      	ldr	r3, [r3, #0]
 80002c8:	4a30      	ldr	r2, [pc, #192]	; (800038c <uart2_rxtx_init+0xd8>)
 80002ca:	f023 0310 	bic.w	r3, r3, #16
 80002ce:	6013      	str	r3, [r2, #0]
	GPIOA->MODER |= (1U<<5);
 80002d0:	4b2e      	ldr	r3, [pc, #184]	; (800038c <uart2_rxtx_init+0xd8>)
 80002d2:	681b      	ldr	r3, [r3, #0]
 80002d4:	4a2d      	ldr	r2, [pc, #180]	; (800038c <uart2_rxtx_init+0xd8>)
 80002d6:	f043 0320 	orr.w	r3, r3, #32
 80002da:	6013      	str	r3, [r2, #0]

	/*set PA2 alternate function type to UART_TX (AF07)*/
	GPIOA->AFR[0] |= (1U<<8);
 80002dc:	4b2b      	ldr	r3, [pc, #172]	; (800038c <uart2_rxtx_init+0xd8>)
 80002de:	6a1b      	ldr	r3, [r3, #32]
 80002e0:	4a2a      	ldr	r2, [pc, #168]	; (800038c <uart2_rxtx_init+0xd8>)
 80002e2:	f443 7380 	orr.w	r3, r3, #256	; 0x100
 80002e6:	6213      	str	r3, [r2, #32]
	GPIOA->AFR[0] |= (1U<<9);
 80002e8:	4b28      	ldr	r3, [pc, #160]	; (800038c <uart2_rxtx_init+0xd8>)
 80002ea:	6a1b      	ldr	r3, [r3, #32]
 80002ec:	4a27      	ldr	r2, [pc, #156]	; (800038c <uart2_rxtx_init+0xd8>)
 80002ee:	f443 7300 	orr.w	r3, r3, #512	; 0x200
 80002f2:	6213      	str	r3, [r2, #32]
	GPIOA->AFR[0] |= (1U<<10);
 80002f4:	4b25      	ldr	r3, [pc, #148]	; (800038c <uart2_rxtx_init+0xd8>)
 80002f6:	6a1b      	ldr	r3, [r3, #32]
 80002f8:	4a24      	ldr	r2, [pc, #144]	; (800038c <uart2_rxtx_init+0xd8>)
 80002fa:	f443 6380 	orr.w	r3, r3, #1024	; 0x400
 80002fe:	6213      	str	r3, [r2, #32]
	GPIOA->AFR[0] &= ~(1U<<11);
 8000300:	4b22      	ldr	r3, [pc, #136]	; (800038c <uart2_rxtx_init+0xd8>)
 8000302:	6a1b      	ldr	r3, [r3, #32]
 8000304:	4a21      	ldr	r2, [pc, #132]	; (800038c <uart2_rxtx_init+0xd8>)
 8000306:	f423 6300 	bic.w	r3, r3, #2048	; 0x800
 800030a:	6213      	str	r3, [r2, #32]

	/*set PA3 mode to alternate function mode*/
	GPIOA->MODER &= ~(1U<<6);
 800030c:	4b1f      	ldr	r3, [pc, #124]	; (800038c <uart2_rxtx_init+0xd8>)
 800030e:	681b      	ldr	r3, [r3, #0]
 8000310:	4a1e      	ldr	r2, [pc, #120]	; (800038c <uart2_rxtx_init+0xd8>)
 8000312:	f023 0340 	bic.w	r3, r3, #64	; 0x40
 8000316:	6013      	str	r3, [r2, #0]
	GPIOA->MODER |= (1U<<7);
 8000318:	4b1c      	ldr	r3, [pc, #112]	; (800038c <uart2_rxtx_init+0xd8>)
 800031a:	681b      	ldr	r3, [r3, #0]
 800031c:	4a1b      	ldr	r2, [pc, #108]	; (800038c <uart2_rxtx_init+0xd8>)
 800031e:	f043 0380 	orr.w	r3, r3, #128	; 0x80
 8000322:	6013      	str	r3, [r2, #0]

	/*set PA3 alternate function type to UART_RX (AF07)*/
	GPIOA->AFR[0] |= (1U<<12);
 8000324:	4b19      	ldr	r3, [pc, #100]	; (800038c <uart2_rxtx_init+0xd8>)
 8000326:	6a1b      	ldr	r3, [r3, #32]
 8000328:	4a18      	ldr	r2, [pc, #96]	; (800038c <uart2_rxtx_init+0xd8>)
 800032a:	f443 5380 	orr.w	r3, r3, #4096	; 0x1000
 800032e:	6213      	str	r3, [r2, #32]
	GPIOA->AFR[0] |= (1U<<13);
 8000330:	4b16      	ldr	r3, [pc, #88]	; (800038c <uart2_rxtx_init+0xd8>)
 8000332:	6a1b      	ldr	r3, [r3, #32]
 8000334:	4a15      	ldr	r2, [pc, #84]	; (800038c <uart2_rxtx_init+0xd8>)
 8000336:	f443 5300 	orr.w	r3, r3, #8192	; 0x2000
 800033a:	6213      	str	r3, [r2, #32]
	GPIOA->AFR[0] |= (1U<<14);
 800033c:	4b13      	ldr	r3, [pc, #76]	; (800038c <uart2_rxtx_init+0xd8>)
 800033e:	6a1b      	ldr	r3, [r3, #32]
 8000340:	4a12      	ldr	r2, [pc, #72]	; (800038c <uart2_rxtx_init+0xd8>)
 8000342:	f443 4380 	orr.w	r3, r3, #16384	; 0x4000
 8000346:	6213      	str	r3, [r2, #32]
	GPIOA->AFR[0] &= ~(1U<<15);
 8000348:	4b10      	ldr	r3, [pc, #64]	; (800038c <uart2_rxtx_init+0xd8>)
 800034a:	6a1b      	ldr	r3, [r3, #32]
 800034c:	4a0f      	ldr	r2, [pc, #60]	; (800038c <uart2_rxtx_init+0xd8>)
 800034e:	f423 4300 	bic.w	r3, r3, #32768	; 0x8000
 8000352:	6213      	str	r3, [r2, #32]

	/*********configure the uart module *********/
	/*enable clock access to uart2*/
	RCC->APB1ENR |= UART2EN;
 8000354:	4b0c      	ldr	r3, [pc, #48]	; (8000388 <uart2_rxtx_init+0xd4>)
 8000356:	6c1b      	ldr	r3, [r3, #64]	; 0x40
 8000358:	4a0b      	ldr	r2, [pc, #44]	; (8000388 <uart2_rxtx_init+0xd4>)
 800035a:	f443 3300 	orr.w	r3, r3, #131072	; 0x20000
 800035e:	6413      	str	r3, [r2, #64]	; 0x40

	/*configure baudrate*/
	uart_set_baudrate(USART2,APB1_CLK,UART_BAUDRATE);
 8000360:	f44f 32e1 	mov.w	r2, #115200	; 0x1c200
 8000364:	490a      	ldr	r1, [pc, #40]	; (8000390 <uart2_rxtx_init+0xdc>)
 8000366:	480b      	ldr	r0, [pc, #44]	; (8000394 <uart2_rxtx_init+0xe0>)
 8000368:	f000 f892 	bl	8000490 <uart_set_baudrate>

	/*configure the transfer direction*/
	USART2 ->CR1 |= (CR1_TE | CR1_RE);
 800036c:	4b09      	ldr	r3, [pc, #36]	; (8000394 <uart2_rxtx_init+0xe0>)
 800036e:	68db      	ldr	r3, [r3, #12]
 8000370:	4a08      	ldr	r2, [pc, #32]	; (8000394 <uart2_rxtx_init+0xe0>)
 8000372:	f043 030c 	orr.w	r3, r3, #12
 8000376:	60d3      	str	r3, [r2, #12]

	/*enable uart module*/
	USART2 ->CR1 |= CR1_UE;
 8000378:	4b06      	ldr	r3, [pc, #24]	; (8000394 <uart2_rxtx_init+0xe0>)
 800037a:	68db      	ldr	r3, [r3, #12]
 800037c:	4a05      	ldr	r2, [pc, #20]	; (8000394 <uart2_rxtx_init+0xe0>)
 800037e:	f443 5300 	orr.w	r3, r3, #8192	; 0x2000
 8000382:	60d3      	str	r3, [r2, #12]

}
 8000384:	bf00      	nop
 8000386:	bd80      	pop	{r7, pc}
 8000388:	40023800 	.word	0x40023800
 800038c:	40020000 	.word	0x40020000
 8000390:	00f42400 	.word	0x00f42400
 8000394:	40004400 	.word	0x40004400

08000398 <uart2_rx_inerrupt_init>:

void uart2_rx_inerrupt_init(void){
 8000398:	b580      	push	{r7, lr}
 800039a:	af00      	add	r7, sp, #0
	/*********configure the uart gpioa pin*********/
	/*enable clock access to gpioa*/
	RCC->AHB1ENR |= GPIOAEN;
 800039c:	4b38      	ldr	r3, [pc, #224]	; (8000480 <uart2_rx_inerrupt_init+0xe8>)
 800039e:	6b1b      	ldr	r3, [r3, #48]	; 0x30
 80003a0:	4a37      	ldr	r2, [pc, #220]	; (8000480 <uart2_rx_inerrupt_init+0xe8>)
 80003a2:	f043 0301 	orr.w	r3, r3, #1
 80003a6:	6313      	str	r3, [r2, #48]	; 0x30

	/*set PA2 mode to alternate function mode*/
	GPIOA->MODER &= ~(1U<<4);
 80003a8:	4b36      	ldr	r3, [pc, #216]	; (8000484 <uart2_rx_inerrupt_init+0xec>)
 80003aa:	681b      	ldr	r3, [r3, #0]
 80003ac:	4a35      	ldr	r2, [pc, #212]	; (8000484 <uart2_rx_inerrupt_init+0xec>)
 80003ae:	f023 0310 	bic.w	r3, r3, #16
 80003b2:	6013      	str	r3, [r2, #0]
	GPIOA->MODER |= (1U<<5);
 80003b4:	4b33      	ldr	r3, [pc, #204]	; (8000484 <uart2_rx_inerrupt_init+0xec>)
 80003b6:	681b      	ldr	r3, [r3, #0]
 80003b8:	4a32      	ldr	r2, [pc, #200]	; (8000484 <uart2_rx_inerrupt_init+0xec>)
 80003ba:	f043 0320 	orr.w	r3, r3, #32
 80003be:	6013      	str	r3, [r2, #0]

	/*set PA2 alternate function type to UART_TX (AF07)*/
	GPIOA->AFR[0] |= (1U<<8);
 80003c0:	4b30      	ldr	r3, [pc, #192]	; (8000484 <uart2_rx_inerrupt_init+0xec>)
 80003c2:	6a1b      	ldr	r3, [r3, #32]
 80003c4:	4a2f      	ldr	r2, [pc, #188]	; (8000484 <uart2_rx_inerrupt_init+0xec>)
 80003c6:	f443 7380 	orr.w	r3, r3, #256	; 0x100
 80003ca:	6213      	str	r3, [r2, #32]
	GPIOA->AFR[0] |= (1U<<9);
 80003cc:	4b2d      	ldr	r3, [pc, #180]	; (8000484 <uart2_rx_inerrupt_init+0xec>)
 80003ce:	6a1b      	ldr	r3, [r3, #32]
 80003d0:	4a2c      	ldr	r2, [pc, #176]	; (8000484 <uart2_rx_inerrupt_init+0xec>)
 80003d2:	f443 7300 	orr.w	r3, r3, #512	; 0x200
 80003d6:	6213      	str	r3, [r2, #32]
	GPIOA->AFR[0] |= (1U<<10);
 80003d8:	4b2a      	ldr	r3, [pc, #168]	; (8000484 <uart2_rx_inerrupt_init+0xec>)
 80003da:	6a1b      	ldr	r3, [r3, #32]
 80003dc:	4a29      	ldr	r2, [pc, #164]	; (8000484 <uart2_rx_inerrupt_init+0xec>)
 80003de:	f443 6380 	orr.w	r3, r3, #1024	; 0x400
 80003e2:	6213      	str	r3, [r2, #32]
	GPIOA->AFR[0] &= ~(1U<<11);
 80003e4:	4b27      	ldr	r3, [pc, #156]	; (8000484 <uart2_rx_inerrupt_init+0xec>)
 80003e6:	6a1b      	ldr	r3, [r3, #32]
 80003e8:	4a26      	ldr	r2, [pc, #152]	; (8000484 <uart2_rx_inerrupt_init+0xec>)
 80003ea:	f423 6300 	bic.w	r3, r3, #2048	; 0x800
 80003ee:	6213      	str	r3, [r2, #32]

	/*set PA3 mode to alternate function mode*/
	GPIOA->MODER &= ~(1U<<6);
 80003f0:	4b24      	ldr	r3, [pc, #144]	; (8000484 <uart2_rx_inerrupt_init+0xec>)
 80003f2:	681b      	ldr	r3, [r3, #0]
 80003f4:	4a23      	ldr	r2, [pc, #140]	; (8000484 <uart2_rx_inerrupt_init+0xec>)
 80003f6:	f023 0340 	bic.w	r3, r3, #64	; 0x40
 80003fa:	6013      	str	r3, [r2, #0]
	GPIOA->MODER |= (1U<<7);
 80003fc:	4b21      	ldr	r3, [pc, #132]	; (8000484 <uart2_rx_inerrupt_init+0xec>)
 80003fe:	681b      	ldr	r3, [r3, #0]
 8000400:	4a20      	ldr	r2, [pc, #128]	; (8000484 <uart2_rx_inerrupt_init+0xec>)
 8000402:	f043 0380 	orr.w	r3, r3, #128	; 0x80
 8000406:	6013      	str	r3, [r2, #0]

	/*set PA3 alternate function type to UART_RX (AF07)*/
	GPIOA->AFR[0] |= (1U<<12);
 8000408:	4b1e      	ldr	r3, [pc, #120]	; (8000484 <uart2_rx_inerrupt_init+0xec>)
 800040a:	6a1b      	ldr	r3, [r3, #32]
 800040c:	4a1d      	ldr	r2, [pc, #116]	; (8000484 <uart2_rx_inerrupt_init+0xec>)
 800040e:	f443 5380 	orr.w	r3, r3, #4096	; 0x1000
 8000412:	6213      	str	r3, [r2, #32]
	GPIOA->AFR[0] |= (1U<<13);
 8000414:	4b1b      	ldr	r3, [pc, #108]	; (8000484 <uart2_rx_inerrupt_init+0xec>)
 8000416:	6a1b      	ldr	r3, [r3, #32]
 8000418:	4a1a      	ldr	r2, [pc, #104]	; (8000484 <uart2_rx_inerrupt_init+0xec>)
 800041a:	f443 5300 	orr.w	r3, r3, #8192	; 0x2000
 800041e:	6213      	str	r3, [r2, #32]
	GPIOA->AFR[0] |= (1U<<14);
 8000420:	4b18      	ldr	r3, [pc, #96]	; (8000484 <uart2_rx_inerrupt_init+0xec>)
 8000422:	6a1b      	ldr	r3, [r3, #32]
 8000424:	4a17      	ldr	r2, [pc, #92]	; (8000484 <uart2_rx_inerrupt_init+0xec>)
 8000426:	f443 4380 	orr.w	r3, r3, #16384	; 0x4000
 800042a:	6213      	str	r3, [r2, #32]
	GPIOA->AFR[0] &= ~(1U<<15);
 800042c:	4b15      	ldr	r3, [pc, #84]	; (8000484 <uart2_rx_inerrupt_init+0xec>)
 800042e:	6a1b      	ldr	r3, [r3, #32]
 8000430:	4a14      	ldr	r2, [pc, #80]	; (8000484 <uart2_rx_inerrupt_init+0xec>)
 8000432:	f423 4300 	bic.w	r3, r3, #32768	; 0x8000
 8000436:	6213      	str	r3, [r2, #32]

	/*********configure the uart module *********/
	/*enable clock access to uart2*/
	RCC->APB1ENR |= UART2EN;
 8000438:	4b11      	ldr	r3, [pc, #68]	; (8000480 <uart2_rx_inerrupt_init+0xe8>)
 800043a:	6c1b      	ldr	r3, [r3, #64]	; 0x40
 800043c:	4a10      	ldr	r2, [pc, #64]	; (8000480 <uart2_rx_inerrupt_init+0xe8>)
 800043e:	f443 3300 	orr.w	r3, r3, #131072	; 0x20000
 8000442:	6413      	str	r3, [r2, #64]	; 0x40

	/*configure baudrate*/
	uart_set_baudrate(USART2,APB1_CLK,UART_BAUDRATE);
 8000444:	f44f 32e1 	mov.w	r2, #115200	; 0x1c200
 8000448:	490f      	ldr	r1, [pc, #60]	; (8000488 <uart2_rx_inerrupt_init+0xf0>)
 800044a:	4810      	ldr	r0, [pc, #64]	; (800048c <uart2_rx_inerrupt_init+0xf4>)
 800044c:	f000 f820 	bl	8000490 <uart_set_baudrate>

	/*configure the transfer direction*/
	USART2 ->CR1 |= (CR1_TE | CR1_RE);
 8000450:	4b0e      	ldr	r3, [pc, #56]	; (800048c <uart2_rx_inerrupt_init+0xf4>)
 8000452:	68db      	ldr	r3, [r3, #12]
 8000454:	4a0d      	ldr	r2, [pc, #52]	; (800048c <uart2_rx_inerrupt_init+0xf4>)
 8000456:	f043 030c 	orr.w	r3, r3, #12
 800045a:	60d3      	str	r3, [r2, #12]

	/*enable RXNE interrupt*/
	USART2->CR1 |= CR1_RXNEIE;
 800045c:	4b0b      	ldr	r3, [pc, #44]	; (800048c <uart2_rx_inerrupt_init+0xf4>)
 800045e:	68db      	ldr	r3, [r3, #12]
 8000460:	4a0a      	ldr	r2, [pc, #40]	; (800048c <uart2_rx_inerrupt_init+0xf4>)
 8000462:	f043 0320 	orr.w	r3, r3, #32
 8000466:	60d3      	str	r3, [r2, #12]

	/*enable UART2 interrupt in NVIC*/
	NVIC_EnableIRQ(USART2_IRQn);
 8000468:	2026      	movs	r0, #38	; 0x26
 800046a:	f7ff ff05 	bl	8000278 <__NVIC_EnableIRQ>

	/*enable uart module*/
	USART2 ->CR1 |= CR1_UE;
 800046e:	4b07      	ldr	r3, [pc, #28]	; (800048c <uart2_rx_inerrupt_init+0xf4>)
 8000470:	68db      	ldr	r3, [r3, #12]
 8000472:	4a06      	ldr	r2, [pc, #24]	; (800048c <uart2_rx_inerrupt_init+0xf4>)
 8000474:	f443 5300 	orr.w	r3, r3, #8192	; 0x2000
 8000478:	60d3      	str	r3, [r2, #12]

}
 800047a:	bf00      	nop
 800047c:	bd80      	pop	{r7, pc}
 800047e:	bf00      	nop
 8000480:	40023800 	.word	0x40023800
 8000484:	40020000 	.word	0x40020000
 8000488:	00f42400 	.word	0x00f42400
 800048c:	40004400 	.word	0x40004400

08000490 <uart_set_baudrate>:
	while(!(USART2->SR & SR_TXE)){}
	/*write to transmit data register*/
	USART2->DR = (ch & 0xFF);
}

static void uart_set_baudrate(USART_TypeDef *USARTx, uint32_t PeriphClk, uint32_t BaudRate){
 8000490:	b580      	push	{r7, lr}
 8000492:	b084      	sub	sp, #16
 8000494:	af00      	add	r7, sp, #0
 8000496:	60f8      	str	r0, [r7, #12]
 8000498:	60b9      	str	r1, [r7, #8]
 800049a:	607a      	str	r2, [r7, #4]
	USARTx->BRR = compute_uart_bd(PeriphClk, BaudRate);
 800049c:	6879      	ldr	r1, [r7, #4]
 800049e:	68b8      	ldr	r0, [r7, #8]
 80004a0:	f000 f808 	bl	80004b4 <compute_uart_bd>
 80004a4:	4603      	mov	r3, r0
 80004a6:	461a      	mov	r2, r3
 80004a8:	68fb      	ldr	r3, [r7, #12]
 80004aa:	609a      	str	r2, [r3, #8]
}
 80004ac:	bf00      	nop
 80004ae:	3710      	adds	r7, #16
 80004b0:	46bd      	mov	sp, r7
 80004b2:	bd80      	pop	{r7, pc}

080004b4 <compute_uart_bd>:

static uint16_t compute_uart_bd(uint32_t PeriphClk, uint32_t BaudRate){
 80004b4:	b480      	push	{r7}
 80004b6:	b083      	sub	sp, #12
 80004b8:	af00      	add	r7, sp, #0
 80004ba:	6078      	str	r0, [r7, #4]
 80004bc:	6039      	str	r1, [r7, #0]
	return ((PeriphClk + (BaudRate/2U))/BaudRate);
 80004be:	683b      	ldr	r3, [r7, #0]
 80004c0:	085a      	lsrs	r2, r3, #1
 80004c2:	687b      	ldr	r3, [r7, #4]
 80004c4:	441a      	add	r2, r3
 80004c6:	683b      	ldr	r3, [r7, #0]
 80004c8:	fbb2 f3f3 	udiv	r3, r2, r3
 80004cc:	b29b      	uxth	r3, r3
}
 80004ce:	4618      	mov	r0, r3
 80004d0:	370c      	adds	r7, #12
 80004d2:	46bd      	mov	sp, r7
 80004d4:	f85d 7b04 	ldr.w	r7, [sp], #4
 80004d8:	4770      	bx	lr
	...

080004dc <Reset_Handler>:

  .section .text.Reset_Handler
  .weak Reset_Handler
  .type Reset_Handler, %function
Reset_Handler:
  ldr   r0, =_estack
 80004dc:	480d      	ldr	r0, [pc, #52]	; (8000514 <LoopForever+0x2>)
  mov   sp, r0          /* set stack pointer */
 80004de:	4685      	mov	sp, r0
/* Call the clock system intitialization function.*/
  bl  SystemInit
 80004e0:	f3af 8000 	nop.w

/* Copy the data segment initializers from flash to SRAM */
  ldr r0, =_sdata
 80004e4:	480c      	ldr	r0, [pc, #48]	; (8000518 <LoopForever+0x6>)
  ldr r1, =_edata
 80004e6:	490d      	ldr	r1, [pc, #52]	; (800051c <LoopForever+0xa>)
  ldr r2, =_sidata
 80004e8:	4a0d      	ldr	r2, [pc, #52]	; (8000520 <LoopForever+0xe>)
  movs r3, #0
 80004ea:	2300      	movs	r3, #0
  b LoopCopyDataInit
 80004ec:	e002      	b.n	80004f4 <LoopCopyDataInit>

080004ee <CopyDataInit>:

CopyDataInit:
  ldr r4, [r2, r3]
 80004ee:	58d4      	ldr	r4, [r2, r3]
  str r4, [r0, r3]
 80004f0:	50c4      	str	r4, [r0, r3]
  adds r3, r3, #4
 80004f2:	3304      	adds	r3, #4

080004f4 <LoopCopyDataInit>:

LoopCopyDataInit:
  adds r4, r0, r3
 80004f4:	18c4      	adds	r4, r0, r3
  cmp r4, r1
 80004f6:	428c      	cmp	r4, r1
  bcc CopyDataInit
 80004f8:	d3f9      	bcc.n	80004ee <CopyDataInit>

/* Zero fill the bss segment. */
  ldr r2, =_sbss
 80004fa:	4a0a      	ldr	r2, [pc, #40]	; (8000524 <LoopForever+0x12>)
  ldr r4, =_ebss
 80004fc:	4c0a      	ldr	r4, [pc, #40]	; (8000528 <LoopForever+0x16>)
  movs r3, #0
 80004fe:	2300      	movs	r3, #0
  b LoopFillZerobss
 8000500:	e001      	b.n	8000506 <LoopFillZerobss>

08000502 <FillZerobss>:

FillZerobss:
  str  r3, [r2]
 8000502:	6013      	str	r3, [r2, #0]
  adds r2, r2, #4
 8000504:	3204      	adds	r2, #4

08000506 <LoopFillZerobss>:

LoopFillZerobss:
  cmp r2, r4
 8000506:	42a2      	cmp	r2, r4
  bcc FillZerobss
 8000508:	d3fb      	bcc.n	8000502 <FillZerobss>

/* Call static constructors */
  bl __libc_init_array
 800050a:	f000 f811 	bl	8000530 <__libc_init_array>
/* Call the application's entry point.*/
  bl main
 800050e:	f7ff fe63 	bl	80001d8 <main>

08000512 <LoopForever>:

LoopForever:
    b LoopForever
 8000512:	e7fe      	b.n	8000512 <LoopForever>
  ldr   r0, =_estack
 8000514:	20020000 	.word	0x20020000
  ldr r0, =_sdata
 8000518:	20000000 	.word	0x20000000
  ldr r1, =_edata
 800051c:	20000000 	.word	0x20000000
  ldr r2, =_sidata
 8000520:	08000598 	.word	0x08000598
  ldr r2, =_sbss
 8000524:	20000000 	.word	0x20000000
  ldr r4, =_ebss
 8000528:	20000020 	.word	0x20000020

0800052c <ADC_IRQHandler>:
 * @retval : None
*/
  .section .text.Default_Handler,"ax",%progbits
Default_Handler:
Infinite_Loop:
  b Infinite_Loop
 800052c:	e7fe      	b.n	800052c <ADC_IRQHandler>
	...

08000530 <__libc_init_array>:
 8000530:	b570      	push	{r4, r5, r6, lr}
 8000532:	4d0d      	ldr	r5, [pc, #52]	; (8000568 <__libc_init_array+0x38>)
 8000534:	4c0d      	ldr	r4, [pc, #52]	; (800056c <__libc_init_array+0x3c>)
 8000536:	1b64      	subs	r4, r4, r5
 8000538:	10a4      	asrs	r4, r4, #2
 800053a:	2600      	movs	r6, #0
 800053c:	42a6      	cmp	r6, r4
 800053e:	d109      	bne.n	8000554 <__libc_init_array+0x24>
 8000540:	4d0b      	ldr	r5, [pc, #44]	; (8000570 <__libc_init_array+0x40>)
 8000542:	4c0c      	ldr	r4, [pc, #48]	; (8000574 <__libc_init_array+0x44>)
 8000544:	f000 f818 	bl	8000578 <_init>
 8000548:	1b64      	subs	r4, r4, r5
 800054a:	10a4      	asrs	r4, r4, #2
 800054c:	2600      	movs	r6, #0
 800054e:	42a6      	cmp	r6, r4
 8000550:	d105      	bne.n	800055e <__libc_init_array+0x2e>
 8000552:	bd70      	pop	{r4, r5, r6, pc}
 8000554:	f855 3b04 	ldr.w	r3, [r5], #4
 8000558:	4798      	blx	r3
 800055a:	3601      	adds	r6, #1
 800055c:	e7ee      	b.n	800053c <__libc_init_array+0xc>
 800055e:	f855 3b04 	ldr.w	r3, [r5], #4
 8000562:	4798      	blx	r3
 8000564:	3601      	adds	r6, #1
 8000566:	e7f2      	b.n	800054e <__libc_init_array+0x1e>
 8000568:	08000590 	.word	0x08000590
 800056c:	08000590 	.word	0x08000590
 8000570:	08000590 	.word	0x08000590
 8000574:	08000594 	.word	0x08000594

08000578 <_init>:
 8000578:	b5f8      	push	{r3, r4, r5, r6, r7, lr}
 800057a:	bf00      	nop
 800057c:	bcf8      	pop	{r3, r4, r5, r6, r7}
 800057e:	bc08      	pop	{r3}
 8000580:	469e      	mov	lr, r3
 8000582:	4770      	bx	lr

08000584 <_fini>:
 8000584:	b5f8      	push	{r3, r4, r5, r6, r7, lr}
 8000586:	bf00      	nop
 8000588:	bcf8      	pop	{r3, r4, r5, r6, r7}
 800058a:	bc08      	pop	{r3}
 800058c:	469e      	mov	lr, r3
 800058e:	4770      	bx	lr
